:100000006F00F07A000000004A0100004C0100007F
:1000100000000000000000000000000000000000E0
:1000200000000000000000000000000000000000D0
:10003000AC0F000000000000AC0F0000000000004A
:10004000AC0F0000AC0F0000AC0F0000AC0F0000C4
:100050001C060000AC0F0000AC0F0000AC0F00004D
:10006000AC0F0000AC0F0000AC0F0000AC0F0000A4
:10007000AC0F0000AC0F0000AC0F0000AC0F000094
:10008000AC0F0000AC0F0000AC0F0000AC0F000084
:10009000AC0F0000AC0F0000AC0F0000000000002F
:1000A000511126C022C206C4828282441244A24058
:1000B000310182802A86014593F6150091C232955E
:1000C00085810606F5F9828000000000634E050276
:1000D00063C305042E86AA857D5515C285466378BF
:1000E000B6006356C00006068606E36CB6FE014500
:1000F00063E4C500918D558D85820582F5FA828075
:100100008682C93F2E8582823305A04063D70500D1
:10011000B305B040C1B7B305B0408682653F330533
:10012000A0408282868263C70500634905005D376F
:100130002E858282B305B040E35B05FE3305A04007
:10014000513F3305B0408282000001A0B707EFBEE7
:1001500037E700E0938707083CC701A07D15131718
:10016000050141839307F00363EBE700B707002025
:100170009387C701AA9788231375F50F82800145DD
:100180008280EFF2FFF1B7E700E03707100023A00D
:10019000E7180F100000EF00B07513051003EF0013
:1001A000B07737450008130505FCB7040020EF00C1
:1001B000B07A01449384C401B38784008C239307ED
:1001C0001400A6979C2337450008130505FCA207D9
:1001D000DD8D2295EF00D07B090493070004E31D19
:1001E000F4FCEF009072C528B7E700E03707100075
:1001F00023A0E7105DBDEFF2BFEAB7460008370461
:1002000000208147938606FC1304C40113060004F2
:100210003387D7001823B305F40085071377F70F4A
:1002200098A1E397C7FE7C301307F00F6312F70223
:10023000056781471307C75A930600043306F70082
:100240000C223306F40085070CA2E399D7FE153F74
:100250000347F403B707002085461377F70F93870A
:10026000870163E4E60098A389B523800700EDBF0A
:100270009307F5FF1397070141839307F00363EB9F
:10028000E704EFF2FFE1B7070020A1462A84938735
:10029000C7016317D5026395A5028566014793865A
:1002A000C65A13060004B385E6008821B385E7002B
:1002B000050788A1E319C7FEE935EF00301211A840
:1002C000BA9798236387E5008CA3653DA547E306AD
:1002D000F4FEE1BB8280EFF2BFDC23A40184239C07
:1002E0000184A3820184238B0184B7070040DE339D
:1002F0001145C207C1832396F184EF00D05E75B328
:10030000EFF21FDA1C210D477111AA8493F7F70F42
:100310006374B70A18311394870013740430598C2E
:100320009306400713F7470F05046312D702A18B0A
:1003300099C7EF00F01DAC2022851D3F91A02285BA
:10034000313DBC20631EF502EF00901C15A893F709
:10035000C70F130780076395E7023C21228593F7B7
:10036000F70F3EC0E53BB8208247418B9D8B19EBD0
:10037000B820B357F540858B0D83058BE386E7FCEA
:10038000110125B33EC0EF00B0188247B820854464
:10039000B394F400E20493778700E184228591C747
:1003A000753B458D9375F50F41BF4D3B93C4F4FFED
:1003B000E98C93F5F40F49B7E394E5FC13F7070FC5
:1003C00093060007E31ED7FA13F777009546631AE2
:1003D000D7001C313707002093F7F70F2300F700F1
:1003E000A5B793F647009DE2B706002003C50600B7
:1003F0000A0575153A954205418159D1A18B95C7DA
:100400002AC0EF00F0108C30024505BF9146630A08
:10041000D70099466309D7009D462145E312D7F6D8
:10042000F1BF7545E1BF1D45D1BF0D3B9C3019BFE4
:100430008280EFF2FFC6B307C5009C231307F003C9
:1004400093F7F70F6397E708130726006353B7087E
:1004500005062A9618221C2285469354770013F429
:10046000F707631ED400A38D0184238D01842386A6
:100470000186B7070020A38097005521B1A009C4C9
:100480009307F4FF13F4F70FB706002083C6260086
:10049000639D960283C6B1858DEA0DC81305F002EF
:1004A000753909CD05461305F0022386C1867D31D5
:1004B00093162500369506052397A186B7070020D9
:1004C000A3809700238D8184CDB66DF823860186A5
:1004D000F5B713F7070C93060004631AD70693D6F3
:1004E0005740139717009187798B858BD98F138786
:1004F000E7FF1377F70F854593F41600E3F5E5F66C
:10050000014463F7F5009387D7038A0713F4F70FC5
:10051000B707002083C727006397970283C7B18579
:100520009DE31DC01305F002153949D90547130590
:10053000F0022386E1861D31131725003A95060542
:100540002397A186A5BF3DF82386018685BF13F7B3
:10055000070E93060008631AD70213D74740058B8E
:10056000238EE18413D73740058BA381E18613D70F
:100570002740058B2381E18613D71740058BA38085
:10058000E186858B2380F186CDBD13F7070F930697
:10059000000B6315D70213D73740058BA383E18681
:1005A00013D72740058B2383E18613D71740058B8C
:1005B000A382E186858B2382F186C1B59306000A6A
:1005C0006315D70213D73740058BA38FE18413D768
:1005D0002740058B238FE18413D71740058BA38E0B
:1005E000E184858B2384F18649BD13F7C70F9306F9
:1005F000C00EE31BD7EC13073600E357B7EC130725
:1006000016002A97182309062A96139587000C22AC
:1006100013750530598D0505A1397DB57111114549
:1006200022C0EF00702A630D050C1145EF00B02BBE
:10063000B7070040DA339387C1848223420741839E
:100640003304874042044180CD4663FB860A371558
:1006500001409145130505809AA3EF00703E4DE1DE
:10066000096713070771938781846377870023A045
:100670000700239C018469A0984385466305D70A37
:1006800025C38946E315D7FE1386618418221334E7
:1006900014050607598C1374F40F9386418400A245
:1006A000982205071377F70F98A2A146631AD7047B
:1006B000938651849822954563E1E50298229375CB
:1006C000F70F138715001377F70F98A214221387DB
:1006D000018593F6F60F2E9714A3054798C30DA036
:1006E000930600051387818563E086021E23930627
:1006F000900F63E7F6001E238507C207C1831EA380
:10070000024411017300203016232546637AD60077
:10071000894694C32382018423830184A3820184B4
:1007200023100700F1BF9306000563F9860009470F
:1007300098C32382018423830184D9B7238BE18466
:1007400023A00700239CE18465BFEFF27F9513018E
:1007500041FC0545EF003032EF00807E693C2923E3
:10076000854513055002EF00B03885653146138486
:100770000559081093850559EF007054371501404D
:100780000C1013050580EF00F02389450145EF00AB
:10079000702C41469305C4006810EF005052681059
:1007A000EF00F00B930740117C86680085473EC838
:1007B00023070100EF00902C85450545EF003035FB
:1007C000B707002003A54701B7450F00938505240F
:1007D000EFF05F907D15C167FD17E8824C08370583
:1007E00000403ECC231B0100230E0100EF0010341B
:1007F000854537050040EF009048B7070040C233F9
:1008000042044180B7070040DE331307703E818FFA
:10081000C207C1836377F7001304843E420441801A
:10082000852383C7618593F7F70FE9DFB7E700E01A
:100830003707100023A0E7180F10000083C551846C
:10084000814793F4F50F9386018513F6F70F6366DE
:100850009604238B0184A3820184B7E700E0370765
:10086000100023A0E710814681471387F4FF63CE71
:10087000E7027C183E97834787FCE395D7F88947C2
:10088000E3F297F81C821307000793F6070F6397AC
:10089000E602A6854800AD34B5B73386D7000822F6
:1008A00050003E9608A285074DB770183E96034645
:1008B00086FC850793F7F70FB18E55BF93F7070CAA
:1008C000130700086395E70048009D3625BF75456E
:1008D000EFF0DF881375050215C58D47E384F4F248
:1008E0001C8245453EC0EFF07F878247E39CA7F01E
:1008F0009C8249453EC0EFF07F868247E394A7F093
:10090000094611A81C8205453EC0EFF03F8582478D
:100910000546E399A7EEA6854800213EE5B5EFF22E
:100920002FF8B70700204111754583C42700EFF069
:10093000FF82058919C193C4140003C4C18593873C
:10094000C1853EC211C81305100299E013052002AB
:10095000EFF0DF801374F50F03C7018601CB130599
:100960003002EFF0AFFF498C1374F40F03C7118608
:1009700001CB13054002EFF06FFE498C1374F40FA6
:1009800003C7218601CB13055002EFF02FFD498CE0
:100990001374F40F03C7318601CB13056002EFF027
:1009A000EFFB498C1374F40F03C7418601CB130589
:1009B0007002EFF0AFFA498C1374F40F03C751863D
:1009C00001CB13058002EFF06FF9498C1374F40F1B
:1009D00003C7618601CB13059002EFF02FF8498C15
:1009E0001374F40F03C7718601CB1305A002EFF057
:1009F000EFF6498C1374F40F03C7818601CB1305FE
:100A0000B002EFF0AFF5498C1374F40F03C7D18532
:100A100001CB1305C002EFF06FF4498C1374F40F8F
:100A200003C7E18501CB1305D002EFF02FF3498C0A
:100A30001374F40F03C7F18501CB1305E002EFF047
:100A4000EFF1498C1374F40F1376140089453715B0
:100A50000140EF00807F9357144013F61700914533
:100A600037150140EF00607EB7370140938707C01C
:100A7000DE377945C207C1833EC0EFF02FEE8947CC
:100A8000631DF50292479C2395C7824781451384D5
:100A9000170099C0A2850144C205B7340140C18145
:100AA000138504C0EF00302193150401C181138523
:100AB00004C0C1A801448145C5B70945EFF00FEA5C
:100AC00083C6B1859387B1853EC42A840145D1C2CE
:100AD00003C7C18602C209CB13050003EFF00FE87C
:100AE00093170501C1833EC21545EFF02FE7131799
:100AF0000501418319453AC6EFF04FE63247931698
:100B000005010546C1826364E6001307F00F054640
:100B1000636CD600B306874013D5F601369505857C
:100B2000229593160501C182A24705468C23639F37
:100B3000C50492473305F4009307F00F63F4A70050
:100B40001305F00F8245EFF0EFD69305F00FEFF0AD
:100B50006FD8824702473385A740130417009317C5
:100B600005014204C1834180ADC0A28537340140F4
:100B7000130504C03EC0EF0010148247130504C0E3
:100B8000BE85EF00901341016FF02FD21306F003E2
:100B9000636FB600FD1533858640EFF0AFD1930546
:100BA000E003EFF0AFD2229592473E9571B733053F
:100BB000D740938515FC36C4EFF0CFCF9305F003F3
:100BC000EFF0CFD0A2463695C5B7B7340140BE8509
:100BD000138504C0EF00300EA285D1BDEFF24FCCDB
:100BE0002545EFF0AFD7937775000547638AE70691
:100BF00009471304007D638AE7000D471304401F73
:100C00006385E7002164130404D0218911C10580A4
:100C1000B707002083A44701A2852685EFF08FCB7C
:100C2000C167938787DE814563F4A7008D809D456A
:100C3000B73701400546138507C0EF003007A2858E
:100C40002685EFF02FC99305F5FFB7370140C205A0
:100C5000C181138507C0EF00D005D1316FF0EFC41B
:100C60000964130404F455B7EFF28FC3130181FD37
:100C7000854513055003AD2D056585451305058094
:100C8000852D8547C1443EC86C0099473715014002
:100C900026CA7C8623170100352337150140894772
:100CA00061446C00130505807C8622CA212B6C00F0
:100CB00037150140648622CA312337340140930737
:100CC000B05D8A85130504C03EC202C02304010042
:100CD000B12DC167938707062C08130504C03ECCCD
:100CE00002CE02D002D2512D2C08130504C0EF0011
:100CF0002072130504C08545EF00E0798545130592
:100D000004C0EF00C077D93D130181026FF0EFB945
:100D1000EFF20FB9B7070040D6330567B7040040BC
:100D2000C206C18213077738DE30958FC207C183B0
:100D3000E37CF7FE054699453715014039233734E2
:100D400001408355C4C2130404C022858505C20531
:100D5000C181EF00407681452285EF000076D630D4
:100D6000096737060040C206C1821307F7705E327A
:100D7000958FC207C183E37CF7FE55366FF0EFB263
:100D8000EFF20FB29387A1869A23611119C37D17E1
:100D90009AA31387C1861C2389CF9386E1869E225E
:100DA00089CBFD17C207C1839EA281E723000700FC
:100DB000BD3637060020B70700201306260083C57E
:100DC00017001C221387B1853AC06382B70800233D
:100DD00029CC854701440247102363058604938587
:100DE000018796213EC293840187850696A10D4511
:100DF000636386001145EFF06FB6924799C311E126
:100E000009459E200A0563CFA70082479C2363F60D
:100E100087048507024793F7F70F239004001CA36C
:100E2000EFF0FFAF21016FF04FA8938621879E223C
:100E30001305900F8507C207C1839EA2E37BF5F8D7
:100E40000CA223900600EFF09FAD854769B703C45D
:100E5000A185239901868147BDBFFD1765BFEFF2CC
:100E60002FA4371402401C403707FFF8414593E791
:100E700017001CC05C40F98F5CC01C403707F7FEB0
:100E80007D17F98F1CC01C403707FCFF7D17F98FB9
:100E90001CC05C4041777D17F98F5CC0B7079F008D
:100EA0001CC435291C4C93E707021CCCB717014022
:100EB00003A70740938607401377F7F023A0E74086
:100EC00003A707401367070823A0E74089479CCA88
:100ED000B7F7FF1F03C5477D9307F00F6304F500C5
:100EE0007D89F52EB72702409843C176FD16719B88
:100EF00098C398431367170098C3B7170240D843A5
:100F0000D8C3D843758FD8C3D843B7060001D8C318
:100F10009843558F98C3984393166700E3DD06FE08
:100F2000D843B7160240719BD8C3D8431367270034
:100F3000D8C32147DC42B18BE39EE7FE6FF0EF960A
:100F4000EFF20F96371702405C43370400209146BA
:100F5000B18B130444016385D700A1466382D70493
:100F6000B7376E01938707601CC0B7160240DC429A
:100F70000840918313F7F700B707002093874700D5
:100F8000BA978C23DC4293F5F50F93F70708335794
:100F9000B50081E7EFF00F942A8718C06FF0EF904B
:100FA0005C43B777DC02938707C07DBF01A0970140
:100FB00000209381A186138181FE1305000A97F515
:100FC000FF1F9385250417F6FF1F1306A60363FA78
:100FD000C5008322050023A0550011059105E3EA11
:100FE000C5FE170500001305A56097F5FF1F938543
:100FF000650117F6FF1F1306660263FAC500832218
:10100000050023A0550011059105E3EAC5FE17F57B
:10101000FF1F1305A500938581876377B500232003
:1010200005001105E36DB5FEB7220000938202882A
:10103000739002308D427390428097F2FFFF93824B
:1010400062FC93E2320073905230EFF05FE197F26E
:10105000FFFF9382C26F73901234730020305841A7
:10106000032305004C4537060140930706403E9791
:101070009346F3FFB1C583250640F58D2320B64086
:10108000D043F18ED4C31443B3E6660014C31841B1
:1010900090479346F7FF758E90C7D047F18ED4C71F
:1010A000144541466399C6009447D98E94C7D447E6
:1010B000558FD8C78280B6979443558F98C3828046
:1010C0001C43F58F1CC38280B7070140138707407C
:1010D00083A70740584B698F09C77D8D3335A00022
:1010E000828001458280B707014023AAA740828001
:1010F000B707674537270240938737125CC3B79716
:10110000EFCD9387B79A5CC38280372702401C4B90
:1011100093E707081CCB8280B7270240C8C78280AC
:10112000372702405C470545858B91E74847418951
:10113000133515000D058280EFE29FF62A84CD3726
:1011400085476318F50019E0154529A0D13F7D14A6
:10115000C5BF7DD86FE07FF5EFE29FF4AA84370525
:101160000B00D93F91476313F502372402401C4816
:1011700037050B0093E727001CC844C81C4893E7B9
:1011800007041CC8553F1C48F59B1CC86FE0FFF1C5
:10119000EFE21FF17111AA8409652EC0713F9147DA
:1011A0008245631EF500372402401C48096593E719
:1011B00017001CC88EA049371C48F99B1CC8110198
:1011C0006FE0BFEE944593F7060193F2F60081C7F6
:1011D000DC41B3E2F20083D3050093F7F30FA5C31C
:1011E00003230500611122C226C081471304800237
:1011F0009304800405473316F70033F7C3006312E6
:10120000E602939527003D473317B7001347F7FFD2
:1012100033736700B395B20033E36500639D8600C6
:1012200050C985072147E397E7FC12442320650056
:10123000824421018280E39696FE10C9DDB7828048
:1012400008456D8D3335A000828019C20CC982809B
:101250004CC9828037070140144786058D47B397F4
:10126000B70093C7F7FFF58F1CC71C47B315B50030
:10127000DD8D0CC7828023AAA186828083A6418748
:10128000854718216390F6021C31639CD7023C21EC
:101290009A0793E707F8B7E600E093F7F70FBA96D7
:1012A0002380F6408546935757003397E600544114
:1012B00089CE938707048A07B7E600E0B69798C3FC
:1012C0008280EDF33C219A07F9B793870706B7E6CA
:1012D00000E08A07B69798C30F1000008280371786
:1012E00002401C430E0593F777F05D8D08C38280A2
:1012F00099C5371702401C4F5D8D08CF8280B71704
:101300000240984F1345F5FF798D88CF828099C5AB
:10131000371702405C4F5D8D48CF8280B71702407F
:10132000D84F1345F5FF798DC8CF82801E213737FE
:101330000140130707C0C207C1836306E5003707F2
:1013400000406316E500BA2193F7F7F8D98FFA2128
:1013500093F7F7CFC207C183D98F1EA1DE215EB5F7
:101360009E211EB5B7370140938707C06314F5006F
:101370009C251EB985475EA982801E3165771307BB
:10138000F7CFC207C183BD9BC207C1831EB11E3107
:10139000562103D38500C20713960601162DC1837B
:1013A00093F7F7FD758F96214182A206558FB621DE
:1013B00042074183B3E666009206D58FB7360140F7
:1013C000C207938606C0C183631ED502B62593F774
:1013D000F7F703D3C5009206D58FD621C207C18384
:1013E000920693F7F7FBD58FFD769386F63FF18E45
:1013F000F225C207C183336666000A06D18E1396B2
:101400000601418252A11AADFA2118DD1EB1828077
:101410001A31FD77FD17F98F1EB1035305025A21CA
:101420005E2DE5769386F6CFFD8E9E21131607017D
:10143000BA21A207DD8EF977FD17B3F7670003D352
:101440008500C2064182336767003207D98F37377C
:101450000140C207130707C0C182C183631BE500B7
:1014600071777D17718FD2251A06518F13160701D8
:101470004182FA2152A156AD38C11EB182801E218F
:1014800089C593E717001EA18280C207C183F99B1B
:10149000C207C183CDBF8357450491C52167D98F4A
:1014A0002312F5048280C607C583DDBF0EB552A99D
:1014B00082804EB582800CDD82802CC18280B3C7D1
:1014C000A5008D8B3307C50081E78D4763E7C70211
:1014D000AA87637EE50A942185078505A38FD7FE39
:1014E000E3EBE7FE8280942185078505A38FD7FE75
:1014F000E3EBE7FE02441101828093763500AA8770
:1015000089CA942185078505A38FD7FE93F63700F6
:10151000C5BF9376C7FF138606FE63F5C706711134
:1015200022C0C04903A3050083A38500C0CB804D22
:1015300023A0670003A3450080CFC04D23A267000E
:1015400083A2C50003A3050193854502C0CF03A470
:10155000C5FF23A4770023A6570023A8670093871D
:10156000470223AE87FEE3EEC7FAE3F3D7F89041D4
:101570009107910523AEC7FECDBF9041910791051C
:1015800023AEC7FEE3EBD7FEE3E7E7F48280828079
:10159000040000000100000004000000040000003E
:1015A0000000000010000000010000000300000027
:1015B000FF000A9C0040000000000000C080000006
:1015C000000000000000000002000000010204080A
:1015D00010200000000000000000000000000A03CE
:0C15E0000E1400000000000000000000DD
:1015EC0001010100010203040506070801020304BE
:0815FC0005060708006CDC0283
:00000001FF
